:020000040000FA
:0600000023EF01F01200E5
:02002A000000D4
:04002C00D9CFE6FF43
:10003000E1CFD9FF040EE126DE6ADD6ADECF02F0F1
:10004000DDCF03F0D890035004E6880E025C130E57
:1000500003581DE2020EDB6A030EDB6A020EDBCFE1
:1000600002F0030EDBCF03F0D890035004E6020E3B
:10007000025C000E035806E2020EDB2A030E01E3C7
:10008000DB2AECD7DF2A010E01E3DB2AD7D7040EE7
:10009000E15C02E2E16AE552E16EE552E7CFD9FFA9
:1000A0001200D9CFE6FFE1CFD9FF040EE126DE6AC8
:1000B000DD6ADECF02F0DDCF03F0D890035004E616
:1000C000200E025C030E03581DE2020EDB6A030ED3
:1000D000DB6A020EDBCF02F0030EDBCF03F0D89019
:1000E000035004E6020E025C000E035806E2020E04
:1000F000DB2A030E01E3DB2AECD7DF2A010E01E342
:10010000DB2AD7D7040EE15C02E2E16AE552E16E38
:10011000E552E7CFD9FF1200D9CFE6FFE1CFD9FFF3
:10012000020EE126DE6ADD6ADECF02F0DDCF03F0EB
:10013000D890035004E6320E025C000E03580DE224
:100140008C708C50010B02E08C9201D08C82A9DF64
:10015000DF2A010E01E3DB2AE7D7020EE15C02E2AF
:10016000E16AE552E16EE552E7CFD9FF12008A80DD
:100170008A828A848A865ADF8A908A928A948A96A8
:1001800016EF00F0956AF00E936E0F0E8A6E4EDF3A
:100190008A6A4CDF8C708C50010B02E08C9201D08B
:0801A0008C8244DFF2D712004B
:0801A8002A0EF66E000EF76E40
:1001B000000EF86E00010900F550656F0900F5505A
:1001C000666F03E1656701D03DD00900F550606FAF
:1001D0000900F550616F0900F550626F09000900D0
:1001E000F550E96E0900F550EA6E090009000900B2
:1001F000F550636F0900F550646F09000900F6CFF0
:1002000067F0F7CF68F0F8CF69F060C0F6FF61C023
:10021000F7FF62C0F8FF0001635302E1645307E097
:100220000900F550EE6E6307F8E26407F9D767C07E
:10023000F6FF68C0F7FF69C0F8FF00016507000E10
:06024000665BBFD712004F
:0A02460013EE00F023EE00F0F86A5A
:10025000019CD4EC00F031EC01F0C2EC00F0FBD7D3
:0202600012008A
:02026200120088
:020000040030CA
:0100000024DB
:0100010008F6
:0100020019E4
:010003001EDE
:0100050001F9
:010006008178
:010008000FE8
:01000900C036
:01000A000FE6
:01000B00E014
:01000C000FE4
:01000D0040B2
:00000001FF
